:1000000000308A007F2C0000FF00030E8301A10056
:100010000A08A0008A010408A2007708A300780853
:10002000A4007908A5007A08A6007B08A70083131E
:1000300083128C308400001D1F280C1932282208DE
:1000400084002308F7002408F8002508F900260892
:10005000FA002708FB0020088A00210E8300FF0E0B
:100060007F0E09008A110A1235281430AB000C11DA
:100070008A110A121F283F3085008601FF30870051
:1000800088018901203083168500FF3086001F30EB
:1000900087008312DA00FF30831688000910891068
:1000A0000911811383121F0838399F000630831607
:1000B0009F0083129412DA125A0883168700831263
:1000C0005A165A088316870085168312DA155A08BD
:1000D0008316870034308312940000308316940016
:1000E0008312071197010530970083160C15C03055
:1000F00083128B04A801A901AA011430AB008A1154
:100100000A12892C0830F700F70B84288316051291
:10011000831205120330F700F70B8C28831605169F
:10012000831200345A155A08831687008312071960
:100130009228AB012B08033C031CEB2883161418F0
:10014000A32883129E2883121308AC00941314135F
:100150002B08F700F7080319BA28013077020319B2
:10016000C328023077020319C62803307702031927
:10017000CA28D9284230AD002C08803C0319C22877
:100180001430AB00DC285A30AD00DC280808603899
:10019000AD00DC280608AD002F08C23C031DD8289E
:1001A0002C08803C031DD8280230A8001430AB0076
:1001B000DC28FF30AD00DC282D0893002E302B0703
:1001C00084002C08800044302B0784002D08800018
:1001D0008220AB0A9A288A110A129C2C5A155A08B6
:1001E0008316870083120719EE28AB012B08073C02
:1001F000031C5F2983161418FF288312FA28831220
:100200001308AC00941314132B08F700F708031914
:1002100026290130770203192F29023077020319AA
:100220003229033077020319362904307702031983
:1002300039290530770203193C2906307702031962
:100240003F2907307702031942294D29CE30AD00EE
:100250002C08803C03192E291430AB0050295A3049
:10026000AD00502908086038AD0050290608AD00DF
:1002700050290130AD0050290130AD005029013026
:10028000AD0050290130AD002F08C23C031D4C29A0
:100290000230A8001430AB005029FF30AD005029C7
:1002A0002D0893002E302B0784002C08800044304A
:1002B0002B0784002D0880008220AB0AF6288A11C3
:1002C0000A129E2C02302B02FA3E03187F29063EAA
:1002D0008229C030AD007F294030AD007F29A908B8
:1002E000031D7429AD0176298030AD007F2940308F
:1002F000AD007F298030AD007F29AD017F298A11B3
:100300000A12952B0A148A100A11820769296C298E
:100310006F2977297A297D2902302B02FA3E0318AA
:10032000B429063EB729AD01B429AD01B429803006
:10033000AD00B429B108031DA0294030AD00A229A9
:100340008030AD00B429B108031DA829AD01AA2948
:100350008030AD00B429B108031DB1295030AD0083
:10036000B3292830AD00B4298A110A12972B0A1438
:100370008A100A1182079329952997299A29A32976
:10038000AB2902302B02FA3E0318D629063ED929A2
:10039000AD01D629AD01D6294030AD00D629AD0139
:1003A000D6298030AD00D629AD01D6298A110A128E
:1003B000992B0A148A100A118207C829CA29CC2944
:1003C000CF29D129D42902302B02FA3E0318FD2966
:1003D000063E002AAD01FD29AD01FD29AD01FD2933
:1003E000B108031DF6292030AD00F829E030AD003A
:1003F000FD29AD01FD29AD01FD298A110A129B2BB2
:100400000A108A140A118207EA29EC29EE29F02938
:10041000F929FB2902302B02FA3E03182E2A063E48
:100420003C2AAA08031D172AFF30AD00182AAD0187
:100430002E2AAA08031D1F2AFF30AD00212A803072
:10044000AD002E2AFF30AD002E2AFF30AD002E2A3F
:10045000FF30AD002E2AFF30AD002E2AB108031D5B
:10046000382A3208803C031D382A0130AA00392A74
:10047000AA018A110A129D2B0A108A140A118207F6
:10048000112A192A222A252A282A2B2AA908031DDB
:100490005D2A02302B02FA3E03185C2A063E7E2AB1
:1004A000AD015C2AAD015C2AAD015C2AAD015C2A7C
:1004B000AD015C2AAD015C2A7B2A290B602A642AE3
:1004C0002908023C031D7B2A02302B02FA3E031846
:1004D0007B2A063E882AFF30AD007B2AFF30AD0024
:1004E0007B2AC030AD007B2AAD017B2AAD017B2A7F
:1004F0005A30AD007B2A8A110A129F2B0A108A14E7
:100500000A118207502A522A542A562A582A5A2A4D
:100510000A108A140A1182076B2A6E2A712A742A19
:10052000762A782A02302B02FA3E0318A52A063EC4
:10053000B92AAD01A52AAD01A52AAD01A52AAD01B3
:10054000A52AAD01A52AAD01A52AB108031DB62A29
:100550002908FD3E0318B62A033EC32AA801B62A7D
:100560000130A800B62A0330A800B62A8A110A1260
:10057000A12B0A108A140A118207992A9B2A9D2A04
:100580009F2AA12AA32A0A108A140A118207AE2AD6
:10059000B02AB32A02302B02FA3E0318DD2A063EA7
:1005A000EB2AAD01DD2AAD01DD2AAD01DD2AAD0169
:1005B000DD2AAD01DD2AAD01DD2A3108803C031DB5
:1005C000E42A0130A900E82AB108031DE82AA9019C
:1005D0008A110A12A32B0A108A140A118207D12A3F
:1005E000D32AD52AD72AD92ADB2A02302B02FA3E6F
:1005F0000318092B063E0E2BAD01092BAD01092B6B
:10060000AD01092BAD01092BAD01092B5A30AD000D
:10061000092B0230A9008A110A12A52B0A148A1488
:100620000A118207FC2AFE2A002B022B042B062B20
:1006300002302B02FA3E03182D2B063E302BAD0163
:100640002D2BAD012D2B4030AD002D2BAD012D2BD1
:10065000AD012D2B5A30AD002D2B8A110A12A72B7C
:100660000A148A140A1182071F2B212B232B262BF5
:10067000282B2A2B5A155A0883168700831207192C
:100680003A2BAB012B08073C031CBD2B8316141817
:100690004B2B8312462B83121308AC0094131413B4
:1006A000AB08031D5C2BCF30AD002C08803C031938
:1006B0005B2B1430AB00AE2B2B0B612B5A30AD00F3
:1006C000AE2B2B08013C0318AC2B2B08073C031C5A
:1006D000AC2B2F08F700A23077020319942B62305D
:1006E00077020319962BE23077020319982B3230E8
:1006F000770203199A2BB230770203199C2B8230B0
:10070000770203199E2BC23077020319A02B2230E7
:1007100077020319A22BF23077020319A42B0230BF
:1007200077020319A62BA82B6229AB2B8C29AB2BA4
:10073000C129AB2BE329AB2B0A2AAB2B462AAB2BC7
:10074000922AAB2BCA2AAB2BF52AAB2B182BAB2B3F
:10075000FF30AD00AB2BAE2B1430AB002D08930057
:100760002E302B0784002C08800044302B07840097
:100770002D0880008220AB0A422B8A110A12A02C7D
:100780005A155A088316870083120719C02BAB012C
:100790002B08133C031C7C2C83161418D12B8312BA
:1007A000CC2B83121308AC00941314132B08F700FE
:1007B000F7080319282C013077020319312C023075
:1007C00077020319342C033077020319382C0430D4
:1007D000770203193A2C0530770203193D2C0630B5
:1007E00077020319402C073077020319432C083095
:1007F00077020319462C093077020319482C0A3076
:10080000770203194A2C0B30770203194C2C0C3059
:10081000770203194E2C0D3077020319502C0E303D
:1008200077020319522C0F3077020319542C103021
:1008300077020319562C113077020319582C123005
:10084000770203195A2C1330770203195C2C6A2C97
:100850009E30AD002C08803C0319302C1430AB00C6
:100860006D2C5A30AD006D2C08086038AD006D2C31
:100870000608AD000130AD006D2C0130AD006D2CCF
:100880000130AD006D2C0130AD006D2CAD016D2C33
:10089000AD016D2CAD016D2CAD016D2CAD016D2C3C
:1008A000AD016D2CAD016D2CAD016D2CAD016D2C2C
:1008B000AD016D2CAD016D2CAD012F08C23C031DA7
:1008C000692C3108803C031D692C0230A8001430CB
:1008D000AB006D2CFF30AD006D2C2D0893002E3039
:1008E0002B0784002C08800044302B0784002D083F
:1008F00080008220AB0AC82B8A110A12A22C840124
:100900001F308305073083169F00FF308312DA0003
:100910003B282808F700F70803199B2C01307702C1
:1009200003199D2C0230770203199F2C03307702A4
:100930000319A12CA32C9228A42CEE28A42C3A2B2A
:0C094000A42CC02BA42CA42C892C630038
:02400E00723FFF
:00000001FF
